:100000008316003085008600831274280130910029
:1000100001309200013093000130940001309500CE
:100020003D280830910004309200043093000230E3
:100030009400013095003D2840309100203092001E
:100040000830930004309400013095003D280030C2
:10005000910000309200603093001E309400013017
:1000600095003D2800309100003092000030930050
:10007000003094007F3095003D28851400008510E5
:1000800011088600502012088600502013088600B0
:1000900050201408860050201508860050200800C3
:1000A0009B0B502800308600051400000510080046
:1000B000FF309100920093009400950080308C00F6
:1000C0006D28910D1110920D1210930D1310940DB7
:1000D0001410950D1510951F08008C0B7228803098
:1000E0008C0061283D206D28F0308C0006208C0BA0
:1000F000762840308C0011208C0B7B2830308C000F
:100100001C208C0B802820308C0027208C0B85280D
:0E01100080308C0032208C0B8A2858207428F6
:00000001FF
